:1000000024C03EC03DC03CC03BC03AC099C438C0CB
:1000100037C036C035C034C033C032C031C030C044
:100020002FC02EC02DC000C301C302C305C306C329
:1000300007C308C30AC30CC30FC313C3BFC4D7C4C9
:10004000E2C4E7C4F5C4FCC40AC511241FBECFE551
:10005000D4E0DEBFCDBF10E0A0E6B0E0E4E5FBE118
:1000600002C005900D92A83DB107D9F721E0A8ED97
:10007000B0E001C01D92AE32B207E1F73EDA68CDC2
:10008000BFCFA998A898A198A0980895A19A82E0B6
:100090008A95F1F700C00895A09AA19A82E08A9506
:1000A000F1F700C0A09882E08A95F1F700C0A1980E
:1000B00082E08A95F1F700C0089598E0A09A87FF42
:1000C00002C0A19801C0A19A22E02A95F1F700C0D0
:1000D000A09822E02A95F1F700C0880F915071F79F
:1000E000A09AA19882E08A95F1F700C0A09822E03A
:1000F0002A95F1F700C083B38695817081950895A4
:10010000282FA09AA19832E03A95F1F700C0A09864
:1001100082E08A95F1F700C093B391FB882780F9BC
:1001200097E0A09A32E03A95F1F700C0A09832E04B
:100130003A95F1F700C0880F99998160915089F73D
:10014000A09A211102C0A19A01C0A19892E09A95AB
:10015000F1F700C0A09832E03A95F1F700C0089599
:10016000FC01680F791F80E048E1E617F70781F08E
:10017000219198E0322F3827532F517030FD84277A
:100180008695513009F480682695915099F7EDCF06
:100190000895282F20779AE0299F9001112494E058
:1001A000359527959A95E1F78F70820F089520E095
:1001B0008A3018F02F5F8A50FBCF90E1299F900181
:1001C0001124822B0895CF93C82FC3706111C06191
:1001D0004111C0685BDF80ED70DF87E06EDF8C2F40
:1001E0006CDFCF9159CFEF92FF920F931F93CF9374
:1001F000DF93EC018B017A0149DF80ED5EDF80E067
:100200005CDF4ADF43DF81ED58DF81E079DFC1DF6A
:10021000F701808341DF3ADF80ED4FDF81E04DDF82
:100220003BDF34DF81ED49DF81E06ADFB2DFF801D7
:10023000808332DF2BDF80ED40DF82E03EDF2CDF8A
:1002400025DF81ED3ADF81E05BDFA3DF8883982F34
:1002500086FF02C09F7101C09F739883DF91CF9189
:100260001F910F91FF90EF9017CFEF92FF920F9396
:100270001F93CF93DF937C018B01EA0107DF80EDB1
:100280001CDF84E01ADF08DF01DF81ED16DF81E08B
:1002900037DF7FDFF7018083FFDEF8DE80ED0DDFE3
:1002A00085E00BDFF9DEF2DE81ED07DF81E028DF9C
:1002B00070DFF8018083F0DEE9DE80EDFEDE86E0AF
:1002C000FCDEEADEE3DE81EDF8DE81E019DF61DFEE
:1002D0008883DF91CF911F910F91FF90EF90DCCE3B
:1002E0001F93CF93DF9300D0CDB7DEB7182F49838C
:1002F0006A83CCDE80EDE1DE80E0DFDE4981842FA1
:1003000056DFDBDE6A81862F52DFD7DE812F4FDF9B
:10031000805CD3DE0F900F90DF91CF911F91BCCE08
:100320001F93CF93DF9300D0CDB7DEB7182F4A834A
:100330006983ACDE80EDC1DE84E0BFDE812F37DF74
:10034000BCDE6981862F33DFB8DE4A81842F2FDF40
:10035000B4DE0F900F90DF91CF911F919DCE0F9340
:100360001F93CF93DF93EC018B01B80188815CDB95
:1003700088839FEF980F9D3F48F4F8019081983251
:1003800039F0903129F0923281F702C081E001C04A
:1003900080E0DF91CF911F910F9108951F93CF932C
:1003A000DF9300D0CDB7DEB7182F69837A8386DA62
:1003B000F7D969817A81882341F084E4113011F002
:1003C0007DDB01C079DB80E001C082E00F900F90FF
:1003D000DF91CF911F910895EF92FF920F931F939A
:1003E000CF93DF93CDB7DEB727970FB6F894DEBF74
:1003F0000FBECDBF7B01473008F45DC09C01295181
:100400003C4F273F3A4208F056C097FF05C09195F0
:100410008195910901E001C000E010E06AE070E020
:100420005BDB21E0210FE1E0F0E0EC0FFD1FE10FCD
:10043000F11D17FDFA95805D8083862F972F122F6F
:10044000181619065CF3822F022E000C990BE1E0BE
:10045000F0E0EC0FFD1FE80FF91F002329F03DE24B
:10046000308330E06EE21DC03BE2FACF41E0430F43
:100470005FEF520FD701A80FB91FE1E0F0E0EC0FDA
:10048000FD1FE20FF11D27FDFA9520812C935111DC
:1004900006C0F701E40FF11D608342E0430F342FE3
:1004A000252F832F90E027FFE1CFF701E80FF91FF9
:1004B000108280E001C081E027960FB6F894DEBF7D
:1004C0000FBECDBFDF91CF911F910F91FF90EF90A5
:1004D0000895AF92BF92CF92DF92EF92FF920F9367
:1004E0001F93CF93DF93CDB7DEB729970FB6F8945C
:1004F000DEBF0FBECDBFF82E8B0160E070E08EEB4B
:10050000DBDACE0101966C015C0169E0E62EE80EB3
:1005100089DAF50181935F01EE12FACF69E070E0AC
:10052000C6011EDE882311F083E065C02A8130E019
:10053000322F22278981282BF0E1FF120DC02E7F58
:1005400053E0220F331F5A95E1F74F818CE090E082
:10055000841B9109280F391F37FF05C0319521955C
:10056000310961E001C060E0F8E2FF1619F042E2F3
:10057000F4120DC08D818076803231F0803431F0FC
:10058000811105C0287F03C02C7F01C02E7FC901C7
:1005900044E0969587954A95E1F77AE0789FA00127
:1005A000799F500D11242F703327E0E8F2E02E9F41
:1005B000C0012F9F900D3E9F900D1124611101C02D
:1005C0009E5F892F992786958695840F951F6623B0
:1005D00019F09195819591099C012A5D3D4F293033
:1005E000374018F4282F892F02C020ED87E0F8014A
:1005F0002083818380E029960FB6F894DEBF0FBE7A
:10060000CDBFDF91CF911F910F91FF90EF90DF90C1
:10061000CF90BF90AF90089590E08B30910528F572
:10062000FC01ED5EFF4F0994C69817C0C69801C043
:10063000C69A9598969818C0C69808C0C69803C0E0
:10064000C69807C0C69A959A09C0C69A959A02C0DC
:10065000C69A9598969A03C0C69A95989698C79800
:100660000895C69A959A969AC79A0895362F9091AA
:10067000EB00992349F01092140110921501109289
:1006800016011092170126C02AE0622F19DA809312
:100690000A0190930B01832F13DA80930C0190933E
:1006A0000D0180E090E021E0FC01E65FFE4F40811B
:1006B000FC01EC50FF4F3081FC01EC5EFE4F431714
:1006C00011F0208301C0108201968430910561F7FA
:1006D0001092E40081E08093FA000895CF92DF92B7
:1006E000EF92FF920F931F93CF93DF93362F92E0F9
:1006F0009093FA002AE0622FE3D980930A01909345
:100700000B01832FDDD980930C0190930D016FEFC6
:100710007FEF80E090E059E1ECE0F0E020E030E0B5
:10072000A82FEC01C550DF4F6E018B0105501F4F04
:10073000EB01C65FDE4F7E010097B1F4442339F030
:10074000B0910A01B11103C01092FB003DC0B091FD
:10075000C400E9015B9FC00DD11D1124C05ADF4FB9
:10076000B881B093FB0030C0B091C400A43011F147
:10077000E9015B9FC00DD11D1124C05ADF4FB88124
:10078000E601B883A13049F4442339F0E701B88188
:10079000B11103C0E801188217C0B091C400EF0185
:1007A0005B9FC00DD11D1124C05ADF4FB881E801F5
:1007B000B8830AC0EF015B9FC00DD11D1124C05A40
:1007C000DF4FB881B093FE00CFE3DCE92197F1F76A
:1007D00000C000002F5F3F4F31962D30310509F0EA
:1007E000ABCFA43069F0FC01E65FFE4F2081FC0135
:1007F000EC50FF4F2083FC01E85EFE4F1082148214
:10080000DFE7E8E321E0D150E0402040E1F700C01D
:10081000000001966F5F7F4F8530910509F07CCF16
:10082000DF91CF911F910F91FF90EF90DF90CF90CC
:1008300008950F931F93CF93DF93362F92E09093F9
:10084000FA002AE0622F3CD980930A0190930B01B1
:10085000832F36D980930C0190930D0183E090E0B3
:1008600025E039E16CE070E040E050E0EC01C5507B
:10087000DF4FDC01A450BF4FE091C400253061F48C
:100880008A013E9F000D111D1124F801E05AFF4F0F
:10089000E081E093FE0028C02130B9F08A013E9F3C
:1008A000000D111D1124F801E05AFF4FE081E8838B
:1008B000E091C4008B013E9F000D111D1124F80131
:1008C000E05AFF4FE081EC930FC08B013E9F000D7B
:1008D000111D1124F801E05AFF4FE081E093FB0065
:1008E00010921A0110921D01EFE3FCE93197F1F724
:1008F00000C000004F5F5F4F6F5F7F4F4C3051056E
:1009000009F0BACF213041F0FC01E65FFE4F408193
:10091000FC01EC50FF4F4083FFE708E311E0F1508A
:1009200000401040E1F700C0000021500197211164
:1009300099CF1092EB00DF91CF911F910F91089505
:100940001F920F920FB60F9211242F933F934F9344
:100950005F936F937F938F939F93AF93BF93EF9327
:10096000FF93E091F800F0E0EE0FFF1FE853FF4F18
:10097000808191819BBD8ABD88B38E6088BB85B321
:10098000877C85BB90981DBC1CBC8091E2008F5F6A
:100990008093E2008A3F09F077C08091F9008130AE
:1009A00009F072C0E091E0008E2F90E08730910551
:1009B00008F068C0FC01E25EFF4F09948091FF00DF
:1009C0008F5F8093FF009091C500891728F0809178
:1009D000E0008F5F8093E0008091FF008E3309F08C
:1009E00051C08091FF008F5F8093FF004BC08091CA
:1009F00000018F5F809300012091C50090E030E0FE
:100A00002152310911C08091FF0081508093FF0075
:100A100014C0809101018F5F809301012091C50076
:100A200090E030E02C523109821793075CF111C03D
:100A300080910001815080930001811123C009C081
:100A40008091FF008F5F8093FF009091C500891710
:100A5000C8F08091E0008F5F8093E00013C0809128
:100A60000101815080930101811103C081E08093D5
:100A7000E000809101018E3329F4809101018150C1
:100A8000809301011092E2008091F900811108C069
:100A90001092FF0010920001109201011092E000EC
:100AA0008091E3008F5F8093E300823309F044C0BC
:100AB0008091FA00813009F03FC080E090E029E1A8
:100AC000FC01EC5EFE4F30813130E1F4E091C40076
:100AD0003091E4002E9FF0011124E30FF11DE05A44
:100AE000FF4F3081FC01E550FF4F30833091E4002F
:100AF0003C3041F4FC01E65FFE4F3081FC01EC50DC
:100B0000FF4F3083019684309105D1F68091E40047
:100B10008F5F8093E400893160F01092E4001092BE
:100B2000FA00109214011092150110921601109201
:100B300017011092E30014C08091FA00811110C0D7
:100B40008091C5008093FB008091C5008093FC00DC
:100B50008091C5008093FD008091C5008093FE00C8
:100B60008091F80081508093F800863009F054C0DD
:100B70008091E7009091E8008130910511F17CF4BB
:100B8000892BC9F58091FB008093200110922101EF
:100B900010922201109223018091F4002BC0823028
:100BA0009105E1F0039739F58091FE0080932301D0
:100BB0001092200110922101109222018091F700E1
:100BC00019C08091FC0080932101109220011092A5
:100BD0002201109223018091F5000CC08091FD004C
:100BE0008093220110922001109221011092230182
:100BF0008091F60011DD8091E7009091E800019668
:100C0000843091052CF49093E8008093E70004C0B1
:100C10001092E8001092E7008091200190E000908F
:100C2000F80002C0959587950A94E2F780FD909AA6
:100C30008091210190E00090F80002C09595879581
:100C40000A94E2F780FDAD9A8091220190E0009035
:100C5000F80002C0959587950A94E2F780FDAB9A5B
:100C60008091230190E00090F80002C0959587954F
:100C70000A94E2F780FDAC9A8091240190E0009004
:100C8000F80002C0959587950A94E2F780FDC39815
:100C90008091250190E00090F80002C0959587951D
:100CA0000A94E2F780FDC1988091260190E00090BF
:100CB000F80002C0959587950A94E2F780FDC298E6
:100CC0008091F800863049F5E091E500F091E6006A
:100CD000E85EFE4F8081813011F4C09A01C0C09857
:100CE000E091E500F091E600E85EFE4F84818130FE
:100CF00011F4979A01C097988091E5009091E600D1
:100D00000196843091052CF49093E6008093E500E1
:100D100004C01092E6001092E5008091F800811165
:100D20000FC08091FF008093240180910001809387
:100D30002501809101018093260187E08093F800CE
:100D4000FF91EF91BF91AF919F918F917F916F91A3
:100D50005F914F913F912F910F900FBE0F901F9079
:100D6000189582E08093FA00819917C08091DE0087
:100D70008A3048F48091DF00811105C08091DE0047
:100D80008F5F8093DE002FE789EA93E02150804057
:100D90009040E1F700C0000070C08091DE00882321
:100DA00009F467C08091EB008F5F863018F4809360
:100DB000EB0002C01092EB008091EB008330B0F4A6
:100DC0002091F1004AE0822F642F7AD68093F400BC
:100DD0009093F5003091F000832F72D68093F60047
:100DE0009093F70040E0632F822F7ADA8091EB0036
:100DF00083508230B8F42091EE004AE0822F642FB5
:100E00005FD68093F4009093F5003091ED00832F2E
:100E100057D68093F6009093F7004091EC00632F33
:100E2000822F7EDA8091EB00853099F482E0809306
:100E3000F4008093F5004091EC00842F6AE040D6E6
:100E40008093F6009093F7006091ED008091EE00A2
:100E500067DA8091C5008093FB008091C500809384
:100E6000FC008091C5008093FD008091C5008093B7
:100E7000FE001092DF001092DE008091EB008330C4
:100E800009F457C028F4813051F0823069F1089597
:100E9000843009F487C0853009F4ACC00895829984
:100EA0000AC08091F1008F5F883118F48093F100BF
:100EB00002C01092F10083990EC08091F1009FEF63
:100EC000980F9093F100839906C08250873118F0F3
:100ED00087E18093F1009A9904C0839B02C08299B4
:100EE0005BC08091F10049C082990AC08091F000F6
:100EF0008F5F8C3318F48093F00002C01092F000E2
:100F000083990EC08091F0009FEF980F9093F000AE
:100F1000839906C082508B3318F08BE38093F000E6
:100F20009A9904C0839B02C0829962C08091F000AC
:100F300058C0829908C08091EE008F5F803208F01F
:100F400081E08093EE0083990BC08091EE009EEFCC
:100F5000980F9F3110F4815001C08FE18093EE0013
:100F600081E080931A0180931D019A9904C0839BAC
:100F700002C0829911C08091EE006AE0A1D58093F1
:100F8000F4009093F5008091C5008093FB00809160
:100F9000C5008093FC0063C08AE08093FB008093CF
:100FA000FC000895829908C08091ED008F5F8D301C
:100FB00008F081E08093ED0083990BC08091ED00F3
:100FC0009EEF980F9C3010F4815001C08CE080930C
:100FD000ED009A9904C0839B02C0829909C0809158
:100FE000ED006AE06DD58093F6009093F7002FC076
:100FF0008AE044C0829905C08091EC008F5F8093A5
:10100000EC00839905C08091EC0081508093EC0046
:1010100010921A0110921D019A9904C0839B02C07C
:10102000829927C082E08093F4001092F5008091AD
:10103000EC006AE045D58093F6009093F70080912C
:10104000C5008093FB008091C5008093FC008091D7
:10105000C5008093FD008091C5008093FE002FE7BE
:1010600089EA93E0215080409040E1F700C0000001
:1010700008958AE08093FB008093FC008093FD003C
:101080008093FE000895CF93DF93CDB7DEB7299705
:101090000FB6F894DEBF0FBECDBF10D41092C600BD
:1010A0008FEF8987898581110BC08091C6002996B1
:1010B0000FB6F894DEBF0FBECDBFDF91CF9108957C
:1010C0008091C6008111F1CFBE016F5F7F4FCE01CD
:1010D000099645D989858E5F823038F38091C600A4
:1010E000DE01119698E0899FA001112420E030E0F4
:1010F0009D91F901E40FF51FEE5FFE4F90832F5F86
:101100003F4F28303105A1F78F5F8093C600CACFCB
:101110001092FA008091C5008093FB008091C50079
:101120008093FC008091C5008093FD008091C500F4
:101130008093FE008091C600811103C0A4DF8093DC
:10114000C60060E070E081E029D9811116C02FE768
:101150008FE492E1215080409040E1F700C0000010
:101160006EE071E080910201B4D9882331F087EEFE
:1011700093E090930F0180930E0180910E01909166
:101180000F0164E670E0A8D4962F41E0682F892F04
:10119000A5DA81E080931E0108956AE091D4692F59
:1011A000109218011092190110921A0110921B014D
:1011B00010921C0110921D0110921E0110921F012D
:1011C00020E030E090E041E070E0522FFC01022E80
:1011D00002C0F595E7950A94E2F7E0FF0FC02115EC
:1011E000310519F440931D0109C0213019F42093F1
:1011F000190104C0223011F440931C01FB0102C00C
:10120000F595E7955A95E2F7E0FF12C021153105F3
:1012100019F440931F010CC0213019F420931B01D5
:1012200007C0223019F440931E0102C040931A01F6
:101230002F5F3F4F2430310541F608954FEE50E0C7
:1012400060EF70E081EF90E0CED78091EF00A5DFF6
:101250006091F0008091F10009CA1092FA004CEE02
:1012600050E06DEE70E08EEE90E0FFD7A4ECB0E0C1
:1012700011968C911197EBEFF0E0808311968C9191
:101280001197818311968C911197828311968C917D
:10129000838340E06091ED008091EE001FDAE8E189
:1012A000F1E081E08283858308958091DC008130C4
:1012B00041F028F0823081F0833009F10895BEDFDB
:1012C00044C08091E9008F3108F4B8DF8091E900D3
:1012D0008F3181F4C2DF0EC08091E9008F3108F4B4
:1012E000ADDF8091C600882381F18091E9008F31C4
:1012F00009F40EDF8091E900843248F11AC0809130
:10130000E9008F3108F49ADF8091E9008F3109F408
:10131000A4DF9091C6008091E900911103C084324E
:10132000B1F407C0843209F4F3DE8091E900893218
:1013300070F04FEE50E060EF70E081EF90E053D737
:101340006091F0008091F10074DA1092E900089544
:10135000819924C08091DF008F5F8093DF0084310A
:1013600099F4109218011092190110921A0110921A
:101370001B0110921C0110921D0110921E0110926F
:101380001F0181E08093EB002FEF80E792E0215076
:1013900080409040E1F700C0000050C08091DF0025
:1013A000882309F449C08091DF008A3008F044C0E6
:1013B0008091DC008F5F8093DC00843010F010920D
:1013C000DC0082E08093EB008093FA001092E90049
:1013D000109218011092190110921A0110921B011B
:1013E00010921C0110921D0110921E0110921F01FB
:1013F0001092F5008091DC008F5F8093F6001092D0
:10140000FB008091C5008093FC008091C500809313
:10141000FD001092FE006091DC0080E090E08BD334
:101420002FEF84E39CE0215080409040E1F700C022
:10143000000004DF1092EB001092DF00829913C0CD
:101440008091DE008A3028F48091DE008F5F8093E7
:10145000DE002FEF80E792E0215080409040E1F7DE
:1014600000C0000030C08091DE00882351F18091DF
:10147000F9008F5F8093F900833010F01092F9002B
:101480006091F90081E090E056D32FEF80E792E081
:10149000215080409040E1F700C000008091F900A9
:1014A000823079F46091FF0082E090E044D3609153
:1014B000000183E090E03FD36091010184E090E07F
:1014C0003AD31092DE00839913C08091DD008A30F8
:1014D00028F48091DD008F5F8093DD002FEF80E79F
:1014E00092E0215080409040E1F700C00000089554
:1014F0008091DD001092DD00089581B3816E81BB83
:1015000087B38F6C87BB84B3886384BB88B38E60DA
:1015100088BB81E08EBD80E895E29BBD8ABD89B71E
:10152000806189BF87B1876087B987EC86B9C69823
:1015300095989698C798C09897988FE78093FB00E6
:101540008093FC008093FD008093FE001092FF00CA
:10155000109200011092010194D541E061E080E019
:1015600032D64CEE50E06DEE70E08EEE90E07DD61F
:1015700024E041E350E062E370E080E390E0EBD1EF
:1015800082DD8093C6002FEF80E792E021508040FB
:101590009040E1F700C000008091C600882321F050
:1015A00060E070E081E0FAD62FEF80E792E0215012
:1015B00080409040E1F700C0000080E090E0B3D2AE
:1015C0008093DC008091DC00843010F01092DC000D
:1015D0002FEF80E792E0215080409040E1F700C07B
:1015E000000081E090E09FD28093F9002FEF80E728
:1015F00092E0215080409040E1F700C000008091CF
:10160000F900823009F582E090E08DD28093FF00EE
:101610002FEF80E792E0215080409040E1F700C03A
:10162000000083E090E07FD2809300012FEF80E7FD
:1016300092E0215080409040E1F700C0000084E03B
:1016400090E071D2809301012FEF80E792E021506A
:1016500080409040E1F700C0000085E08093C40026
:101660008EE28093C5001092F4001092F5008091F4
:10167000DC008F5F8093F6001092F7001092FB0061
:101680001092FE0082E08093FA0078942FEF80E7BA
:1016900092E0215080409040E1F700C00000CEDD94
:1016A0002FEF84E39CE0215080409040E1F700C0A0
:1016B0000000C7ECD7ED1FE701E084E6F82E92E0CA
:1016C000E92E29E4D22E33E0C32E4EE2B42E8091CF
:1016D000EB00811101C03CDE8091EB00811141DB08
:1016E0009A9B5BC08091EB00811157C08091EA000A
:1016F0008111EDCFDADDC6B9349BFECFD6B984B106
:1017000095B19093F3008093F2008091F200909154
:10171000F300803991402CF4C092C400B092C5000F
:1017200031C08091F2009091F3008139914064F0D2
:101730008091F2009091F300843F91402CF4E0926C
:10174000C400D092C5001EC08091F2009091F300B9
:10175000853F914064F08091F2009091F3008835CC
:1017600092402CF40093C400F092C5000BC080910D
:10177000F2009091F3008935924024F01092C40059
:101780001093C5008091E9008F5F8093E9008091FC
:10179000EA008F5F8093EA009ACF1092EA0097CF19
:1017A000E0912A01F0912B019081809129018923F8
:1017B0000895E0912701F0912801908180912901FD
:1017C000892B8083E0912C01F0912D0190818091F3
:1017D0002901892B808308951F93CF93DF931F9254
:1017E000CDB7DEB71FB7F894E0912701F09128013B
:1017F000208190912901909592239083E0912C0172
:10180000F0912D01208190912901922B908395E0F8
:101810009A95F1F70000882399F0E0912C01F0915E
:101820002D01208190912901909592239083E09140
:101830002701F0912801208190912901922B90831A
:1018400090E29A95F1F7E0912A01F0912B01208125
:1018500090912901922309F480E095E79A95F1F798
:101860000000E0912701F091280120819091290149
:10187000922B9083E0912C01F0912D012081909189
:101880002901909592239083662319F0898391DF33
:1018900089811FBF9AE19A95F1F700C00F90DF91FF
:1018A000CF911F910895E0912C01F0912D0190812D
:1018B000809129018095892380830895E0912701F3
:1018C000F09128019081809129018095892380835E
:1018D000E0912C01F0912D01908180912901892BBB
:1018E00080838FEB93E00197F1F700C000003FB7D2
:1018F000F894E0912C01F0912D01908180912901C3
:10190000809589238083E0912701F09128019081BF
:1019100080912901892B80839AEA9A95F1F700C07A
:10192000E0912A01F0912B012081809129013FBF94
:10193000EFE3F3E03197F1F700C00000E0912A01F6
:10194000F0912B01308190912901932311F0822392
:10195000089581E0089550932D0140932C017093D8
:1019600028016093270190932B0180932A0181E045
:1019700001C0880F2A95EAF7809329019FCF60E084
:1019800081702ACFCF93DF93C82FD8E08C2F81703E
:10199000F6DFC6958111C068D150C1F78C2FDF9159
:1019A000CF910895CF93DF93C82FD8E08C2F81700B
:1019B000D13011F060E001C061E00EDFC695811109
:1019C000C068D15099F78C2FDF91CF910895EF9295
:1019D000FF920F931F93CF93DF93182FEB01042FE8
:1019E0006DDF209761F085E5CDDF7E0188E0E80EB0
:1019F000F11C8991C7DFCE15DF05D9F702C08CEC49
:101A0000C1DF812F002339F0DF91CF911F910F911A
:101A1000FF90EF90C7CFDF91CF911F910F91FF9073
:101A2000EF90B0CF8FEFAECFDF92EF92FF920F9398
:101A30001F93CF93DF93E82E8B0140DF811131C0DC
:101A400080EFA0DFD0E0C0E488EFD82EDC0E81E08C
:101A500096DFF82E81E093DF882319F0FF2071F0E4
:101A600022C0F1100BC0CE1530F0F801808180FF4C
:101A700005C0EC1619F0DC2FFF24F3948F2D7FDFC7
:101A8000F80190819695FF2011F09068F8019083FD
:101A9000C150CD11DCCF0F5F1F4FC111D5CF8D2F9E
:101AA00003C08FEF01C08EEFDF91CF911F910F9197
:101AB000FF90EF90DF90089540E089CF41E087CF1D
:101AC000991B79E004C0991F961708F0961B881F90
:101AD0007A95C9F78095089597FB072E16F4009420
:101AE00006D077FD08D00BD007FC05D03EF49095CA
:101AF00081959F4F0895709561957F4F0895AA1B1A
:101B0000BB1B51E107C0AA1FBB1FA617B70710F0E8
:101B1000A61BB70B881F991F5A95A9F7809590951A
:101B2000BC01CD010895E199FECF9FBB8EBBE09A29
:101B300099278DB30895262FE199FECF9FBB8EBBC9
:101B40002DBB0FB6F894E29AE19A0FBE0196089564
:041B5000F894FFCF37
:101B54007F6F655B51473D33291F150B010B151F23
:101B640029333D47515B656F7F645D423B342D26CD
:101B74001F18110A0301030A11181F262D343B42B2
:101B84005D6449423B352F29231D17110B050105BF
:101B94000B11171D23292F353B42492E2A26221EBD
:101BA4001A16120E0A06020102060A0E12161A1E4E
:101BB40022262A2E017F01014B0096002C015B0294
:081BC400B0046009C012802585
:00000001FF
